

Microchip MPLAB XC8 Assembler V2.32 build 20210201212658 
                                                                                               Wed Jan 19 10:39:02 2022

Microchip MPLAB XC8 C Compiler v2.32 (Free license) build 20210201212658 Og1 
     1                           	processor	18F4580
     2                           	fnconf	rparam,??,?,0
     3                           	pagewidth 120
     4                           	opt	flic
     5                           	psect	cinit,global,reloc=2,class=CODE,delta=1
     6                           	psect	cstackCOMRAM,global,class=COMRAM,space=1,delta=1,lowdata,noexec
     7                           	psect	text0,global,reloc=2,class=CODE,delta=1
     8                           	psect	text1,global,reloc=2,class=CODE,delta=1
     9                           	psect	text2,global,reloc=2,class=CODE,delta=1
    10                           	psect	text3,global,reloc=2,class=CODE,delta=1
    11                           	psect	text4,global,reloc=2,class=CODE,delta=1,group=1
    12                           	psect	text5,global,reloc=2,class=CODE,delta=1,group=1
    13                           	psect	intsave_regs,global,class=BIGRAM,space=1,delta=1,noexec
    14                           	psect	rparam,global,class=COMRAM,space=1,delta=1,noexec
    15                           	psect	idloc,global,abs,ovrld,class=IDLOC,space=5,delta=1,noexec
    16                           	psect	config,global,abs,ovrld,class=CONFIG,space=4,delta=1,noexec
    17  0000                     
    18                           ; Version 2.40
    19                           ; Generated 17/11/2021 GMT
    20                           ; 
    21                           ; Copyright © 2021, Microchip Technology Inc. and its subsidiaries ("Microchip")
    22                           ; All rights reserved.
    23                           ; 
    24                           ; This software is developed by Microchip Technology Inc. and its subsidiaries ("Microch
      +                          ip").
    25                           ; 
    26                           ; Redistribution and use in source and binary forms, with or without modification, are
    27                           ; permitted provided that the following conditions are met:
    28                           ; 
    29                           ;     1. Redistributions of source code must retain the above copyright notice, this lis
      +                          t of
    30                           ;        conditions and the following disclaimer.
    31                           ; 
    32                           ;     2. Redistributions in binary form must reproduce the above copyright notice, this 
      +                          list
    33                           ;        of conditions and the following disclaimer in the documentation and/or other
    34                           ;        materials provided with the distribution. Publication is not required when
    35                           ;        this file is used in an embedded application.
    36                           ; 
    37                           ;     3. Microchip's name may not be used to endorse or promote products derived from th
      +                          is
    38                           ;        software without specific prior written permission.
    39                           ; 
    40                           ; THIS SOFTWARE IS PROVIDED BY MICROCHIP "AS IS" AND ANY EXPRESS OR IMPLIED WARRANTIES,
    41                           ; INCLUDING, BUT NOT LIMITED TO, THE IMPLIED WARRANTIES OF MERCHANTABILITY AND FITNESS F
      +                          OR
    42                           ; PURPOSE ARE DISCLAIMED.  IN NO EVENT SHALL MICROCHIP BE LIABLE FOR ANY DIRECT, INDIREC
      +                          T,
    43                           ; INCIDENTAL, SPECIAL, EXEMPLARY, OR CONSEQUENTIAL DAMAGES (INCLUDING BUT NOT LIMITED TO
    44                           ; PROCUREMENT OF SUBSTITUTE GOODS OR SERVICES; LOSS OF USE, DATA OR PROFITS; OR BUSINESS
    45                           ; INTERRUPTION) HOWSOEVER CAUSED AND ON ANY THEORY OF LIABILITY, WHETHER IN CONTRACT, ST
      +                          RICT
    46                           ; LIABILITY, OR TORT (INCLUDING NEGLIGENCE OR OTHERWISE) ARISING IN ANY WAY OUT OF THE U
      +                          SE OF
    47                           ; THIS SOFTWARE, EVEN IF ADVISED OF THE POSSIBILITY OF SUCH DAMAGE.
    48                           ; 
    49                           ; 
    50                           ; Code-generator required, PIC18F4580 Definitions
    51                           ; 
    52                           ; SFR Addresses
    53  0000                     _PORTD	set	3971
    54  0000                     _ADRESH	set	4036
    55  0000                     _ADRESL	set	4035
    56  0000                     _TRISA	set	3986
    57  0000                     _TRISD	set	3989
    58  0000                     _TRISC	set	3988
    59  0000                     _TRISB	set	3987
    60  0000                     _ADCON2	set	4032
    61  0000                     _ADCON1	set	4033
    62  0000                     _ADCON0	set	4034
    63  0000                     _RC1	set	31761
    64  0000                     _RC0	set	31760
    65  0000                     _GODONE	set	32273
    66                           
    67                           ; #config settings
    68                           
    69                           	psect	cinit
    70  007B82                     __pcinit:
    71                           	callstack 0
    72  007B82                     start_initialization:
    73                           	callstack 0
    74  007B82                     __initialization:
    75                           	callstack 0
    76  007B82                     end_of_initialization:
    77                           	callstack 0
    78  007B82                     __end_of__initialization:
    79                           	callstack 0
    80  007B82  0100               	movlb	0
    81  007B84  EFBC  F03E         	goto	_main	;jump to C main() function
    82                           
    83                           	psect	cstackCOMRAM
    84  000001                     __pcstackCOMRAM:
    85                           	callstack 0
    86  000001                     ?___awdiv:
    87                           	callstack 0
    88  000001                     ?___awmod:
    89                           	callstack 0
    90  000001                     delay@ms:
    91                           	callstack 0
    92  000001                     ___awdiv@dividend:
    93                           	callstack 0
    94  000001                     ___awmod@dividend:
    95                           	callstack 0
    96                           
    97                           ; 2 bytes @ 0x0
    98  000001                     	ds	2
    99  000003                     ??_delay:
   100  000003                     ___awdiv@divisor:
   101                           	callstack 0
   102  000003                     ___awmod@divisor:
   103                           	callstack 0
   104                           
   105                           ; 2 bytes @ 0x2
   106  000003                     	ds	1
   107  000004                     delay@i:
   108                           	callstack 0
   109                           
   110                           ; 2 bytes @ 0x3
   111  000004                     	ds	1
   112  000005                     ___awdiv@counter:
   113                           	callstack 0
   114  000005                     ___awmod@counter:
   115                           	callstack 0
   116                           
   117                           ; 1 bytes @ 0x4
   118  000005                     	ds	1
   119  000006                     data@b:
   120                           	callstack 0
   121  000006                     command@c:
   122                           	callstack 0
   123  000006                     ___awdiv@sign:
   124                           	callstack 0
   125  000006                     ___awmod@sign:
   126                           	callstack 0
   127                           
   128                           ; 1 bytes @ 0x5
   129  000006                     	ds	1
   130  000007                     ___awdiv@quotient:
   131                           	callstack 0
   132                           
   133                           ; 2 bytes @ 0x6
   134  000007                     	ds	2
   135  000009                     ??_main:
   136                           
   137                           ; 1 bytes @ 0x8
   138  000009                     	ds	2
   139  00000B                     main@x:
   140                           	callstack 0
   141                           
   142                           ; 2 bytes @ 0xA
   143  00000B                     	ds	2
   144  00000D                     main@p:
   145                           	callstack 0
   146                           
   147                           ; 2 bytes @ 0xC
   148  00000D                     	ds	2
   149  00000F                     main@r:
   150                           	callstack 0
   151                           
   152                           ; 2 bytes @ 0xE
   153  00000F                     	ds	2
   154  000011                     main@s:
   155                           	callstack 0
   156                           
   157                           ; 2 bytes @ 0x10
   158  000011                     	ds	2
   159  000013                     main@a:
   160                           	callstack 0
   161                           
   162                           ; 2 bytes @ 0x12
   163  000013                     	ds	2
   164  000015                     main@q:
   165                           	callstack 0
   166                           
   167                           ; 2 bytes @ 0x14
   168  000015                     	ds	2
   169  000017                     main@y:
   170                           	callstack 0
   171                           
   172                           ; 2 bytes @ 0x16
   173  000017                     	ds	2
   174                           
   175 ;;
   176 ;;Main: autosize = 0, tempsize = 2, incstack = 0, save=0
   177 ;;
   178 ;; *************** function _main *****************
   179 ;; Defined at:
   180 ;;		line 6 in file "ADC.c"
   181 ;; Parameters:    Size  Location     Type
   182 ;;		None
   183 ;; Auto vars:     Size  Location     Type
   184 ;;  y               2   22[COMRAM] int 
   185 ;;  q               2   20[COMRAM] int 
   186 ;;  a               2   18[COMRAM] int 
   187 ;;  s               2   16[COMRAM] int 
   188 ;;  r               2   14[COMRAM] int 
   189 ;;  p               2   12[COMRAM] int 
   190 ;;  x               2   10[COMRAM] int 
   191 ;; Return value:  Size  Location     Type
   192 ;;                  1    wreg      void 
   193 ;; Registers used:
   194 ;;		wreg, status,2, status,0, cstack
   195 ;; Tracked objects:
   196 ;;		On entry : 0/0
   197 ;;		On exit  : 0/0
   198 ;;		Unchanged: 0/0
   199 ;; Data sizes:     COMRAM   BANK0   BANK1   BANK2   BANK3   BANK4   BANK5
   200 ;;      Params:         0       0       0       0       0       0       0
   201 ;;      Locals:        14       0       0       0       0       0       0
   202 ;;      Temps:          2       0       0       0       0       0       0
   203 ;;      Totals:        16       0       0       0       0       0       0
   204 ;;Total ram usage:       16 bytes
   205 ;; Hardware stack levels required when called: 2
   206 ;; This function calls:
   207 ;;		___awdiv
   208 ;;		___awmod
   209 ;;		_command
   210 ;;		_data
   211 ;;		_delay
   212 ;; This function is called by:
   213 ;;		Startup code after reset
   214 ;; This function uses a non-reentrant model
   215 ;;
   216                           
   217                           	psect	text0
   218  007D78                     __ptext0:
   219                           	callstack 0
   220  007D78                     _main:
   221                           	callstack 29
   222  007D78                     
   223                           ;ADC.c: 7:     int a,x=1234,y=0,p,q,r,s;
   224  007D78  0E04               	movlw	4
   225  007D7A  6E0C               	movwf	(main@x+1)^0,c
   226  007D7C  0ED2               	movlw	210
   227  007D7E  6E0B               	movwf	main@x^0,c
   228                           
   229                           ;ADC.c: 8:     ADCON0=0x01;
   230  007D80  0E01               	movlw	1
   231  007D82  6EC2               	movwf	194,c	;volatile
   232                           
   233                           ;ADC.c: 9:     ADCON1=0x0D;
   234  007D84  0E0D               	movlw	13
   235  007D86  6EC1               	movwf	193,c	;volatile
   236                           
   237                           ;ADC.c: 10:     ADCON2=0x86;
   238  007D88  0E86               	movlw	134
   239  007D8A  6EC0               	movwf	192,c	;volatile
   240                           
   241                           ;ADC.c: 11:     TRISB=0x00;
   242  007D8C  0E00               	movlw	0
   243  007D8E  6E93               	movwf	147,c	;volatile
   244                           
   245                           ;ADC.c: 12:     TRISC=0x00;
   246  007D90  0E00               	movlw	0
   247  007D92  6E94               	movwf	148,c	;volatile
   248                           
   249                           ;ADC.c: 13:     TRISD=0x00;
   250  007D94  0E00               	movlw	0
   251  007D96  6E95               	movwf	149,c	;volatile
   252  007D98                     
   253                           ;ADC.c: 14:     TRISA=0xFF;
   254  007D98  6892               	setf	146,c	;volatile
   255  007D9A                     
   256                           ;ADC.c: 15:     command(0x38);
   257  007D9A  0E38               	movlw	56
   258  007D9C  ECC4  F03D         	call	_command
   259  007DA0                     
   260                           ;ADC.c: 16:     command(0x80);
   261  007DA0  0E80               	movlw	128
   262  007DA2  ECC4  F03D         	call	_command
   263  007DA6                     
   264                           ;ADC.c: 17:     command(0x0f);
   265  007DA6  0E0F               	movlw	15
   266  007DA8  ECC4  F03D         	call	_command
   267  007DAC                     
   268                           ;ADC.c: 18:     command(0x06);
   269  007DAC  0E06               	movlw	6
   270  007DAE  ECC4  F03D         	call	_command
   271  007DB2                     
   272                           ;ADC.c: 19:     command(0x01);
   273  007DB2  0E01               	movlw	1
   274  007DB4  ECC4  F03D         	call	_command
   275  007DB8                     l1029:
   276                           
   277                           ;ADC.c: 22:         ADCON0=0x05;
   278  007DB8  0E05               	movlw	5
   279  007DBA  6EC2               	movwf	194,c	;volatile
   280                           
   281                           ;ADC.c: 23:         command(0x80);
   282  007DBC  0E80               	movlw	128
   283  007DBE  ECC4  F03D         	call	_command
   284  007DC2                     
   285                           ;ADC.c: 24:         GODONE=1;
   286  007DC2  82C2               	bsf	4034,1,c	;volatile
   287  007DC4                     l38:
   288  007DC4  B2C2               	btfsc	4034,1,c	;volatile
   289  007DC6  EFE7  F03E         	goto	u281
   290  007DCA  EFE9  F03E         	goto	u280
   291  007DCE                     u281:
   292  007DCE  EFE2  F03E         	goto	l38
   293  007DD2                     u280:
   294  007DD2                     
   295                           ;ADC.c: 26:         a=ADRESL;
   296  007DD2  CFC3 F013          	movff	4035,main@a	;volatile
   297  007DD6  6A14               	clrf	(main@a+1)^0,c
   298  007DD8                     
   299                           ;ADC.c: 27:         a|=(ADRESH<<8);
   300  007DD8  50C4               	movf	196,w,c	;volatile
   301  007DDA  6E0A               	movwf	(??_main+1)^0,c
   302  007DDC  6A09               	clrf	??_main^0,c
   303  007DDE  5009               	movf	??_main^0,w,c
   304  007DE0  1213               	iorwf	main@a^0,f,c
   305  007DE2  500A               	movf	(??_main+1)^0,w,c
   306  007DE4  1214               	iorwf	(main@a+1)^0,f,c
   307  007DE6                     
   308                           ;ADC.c: 28:         p=a/1000;
   309  007DE6  C013  F001         	movff	main@a,___awdiv@dividend
   310  007DEA  C014  F002         	movff	main@a+1,___awdiv@dividend+1
   311  007DEE  0E03               	movlw	3
   312  007DF0  6E04               	movwf	(___awdiv@divisor+1)^0,c
   313  007DF2  0EE8               	movlw	232
   314  007DF4  6E03               	movwf	___awdiv@divisor^0,c
   315  007DF6  EC5A  F03E         	call	___awdiv	;wreg free
   316  007DFA  C001  F00D         	movff	?___awdiv,main@p
   317  007DFE  C002  F00E         	movff	?___awdiv+1,main@p+1
   318  007E02                     
   319                           ;ADC.c: 29:         data(p+48);
   320  007E02  500D               	movf	main@p^0,w,c
   321  007E04  0F30               	addlw	48
   322  007E06  ECD7  F03D         	call	_data
   323  007E0A                     
   324                           ;ADC.c: 30:         delay(1000000);
   325  007E0A  0E42               	movlw	66
   326  007E0C  6E02               	movwf	(delay@ms+1)^0,c
   327  007E0E  0E40               	movlw	64
   328  007E10  6E01               	movwf	delay@ms^0,c
   329  007E12  ECEA  F03D         	call	_delay	;wreg free
   330  007E16                     
   331                           ;ADC.c: 31:         q=(a%1000);
   332  007E16  C013  F001         	movff	main@a,___awmod@dividend
   333  007E1A  C014  F002         	movff	main@a+1,___awmod@dividend+1
   334  007E1E  0E03               	movlw	3
   335  007E20  6E04               	movwf	(___awmod@divisor+1)^0,c
   336  007E22  0EE8               	movlw	232
   337  007E24  6E03               	movwf	___awmod@divisor^0,c
   338  007E26  EC02  F03E         	call	___awmod	;wreg free
   339  007E2A  C001  F015         	movff	?___awmod,main@q
   340  007E2E  C002  F016         	movff	?___awmod+1,main@q+1
   341  007E32                     
   342                           ;ADC.c: 32:         y=q;
   343  007E32  C015  F017         	movff	main@q,main@y
   344  007E36  C016  F018         	movff	main@q+1,main@y+1
   345  007E3A                     
   346                           ;ADC.c: 33:         q=q/100;
   347  007E3A  C015  F001         	movff	main@q,___awdiv@dividend
   348  007E3E  C016  F002         	movff	main@q+1,___awdiv@dividend+1
   349  007E42  0E00               	movlw	0
   350  007E44  6E04               	movwf	(___awdiv@divisor+1)^0,c
   351  007E46  0E64               	movlw	100
   352  007E48  6E03               	movwf	___awdiv@divisor^0,c
   353  007E4A  EC5A  F03E         	call	___awdiv	;wreg free
   354  007E4E  C001  F015         	movff	?___awdiv,main@q
   355  007E52  C002  F016         	movff	?___awdiv+1,main@q+1
   356  007E56                     
   357                           ;ADC.c: 34:         data(q+48);
   358  007E56  5015               	movf	main@q^0,w,c
   359  007E58  0F30               	addlw	48
   360  007E5A  ECD7  F03D         	call	_data
   361  007E5E                     
   362                           ;ADC.c: 36:         y=(y%100);
   363  007E5E  C017  F001         	movff	main@y,___awmod@dividend
   364  007E62  C018  F002         	movff	main@y+1,___awmod@dividend+1
   365  007E66  0E00               	movlw	0
   366  007E68  6E04               	movwf	(___awmod@divisor+1)^0,c
   367  007E6A  0E64               	movlw	100
   368  007E6C  6E03               	movwf	___awmod@divisor^0,c
   369  007E6E  EC02  F03E         	call	___awmod	;wreg free
   370  007E72  C001  F017         	movff	?___awmod,main@y
   371  007E76  C002  F018         	movff	?___awmod+1,main@y+1
   372  007E7A                     
   373                           ;ADC.c: 37:         s=y;
   374  007E7A  C017  F011         	movff	main@y,main@s
   375  007E7E  C018  F012         	movff	main@y+1,main@s+1
   376  007E82                     
   377                           ;ADC.c: 38:         y=y/10;
   378  007E82  C017  F001         	movff	main@y,___awdiv@dividend
   379  007E86  C018  F002         	movff	main@y+1,___awdiv@dividend+1
   380  007E8A  0E00               	movlw	0
   381  007E8C  6E04               	movwf	(___awdiv@divisor+1)^0,c
   382  007E8E  0E0A               	movlw	10
   383  007E90  6E03               	movwf	___awdiv@divisor^0,c
   384  007E92  EC5A  F03E         	call	___awdiv	;wreg free
   385  007E96  C001  F017         	movff	?___awdiv,main@y
   386  007E9A  C002  F018         	movff	?___awdiv+1,main@y+1
   387  007E9E                     
   388                           ;ADC.c: 39:         data(y+48);
   389  007E9E  5017               	movf	main@y^0,w,c
   390  007EA0  0F30               	addlw	48
   391  007EA2  ECD7  F03D         	call	_data
   392  007EA6                     
   393                           ;ADC.c: 41:         r=(s%10);
   394  007EA6  C011  F001         	movff	main@s,___awmod@dividend
   395  007EAA  C012  F002         	movff	main@s+1,___awmod@dividend+1
   396  007EAE  0E00               	movlw	0
   397  007EB0  6E04               	movwf	(___awmod@divisor+1)^0,c
   398  007EB2  0E0A               	movlw	10
   399  007EB4  6E03               	movwf	___awmod@divisor^0,c
   400  007EB6  EC02  F03E         	call	___awmod	;wreg free
   401  007EBA  C001  F00F         	movff	?___awmod,main@r
   402  007EBE  C002  F010         	movff	?___awmod+1,main@r+1
   403  007EC2                     
   404                           ;ADC.c: 43:         data(r+48);
   405  007EC2  500F               	movf	main@r^0,w,c
   406  007EC4  0F30               	addlw	48
   407  007EC6  ECD7  F03D         	call	_data
   408  007ECA                     
   409                           ;ADC.c: 44:         x++;
   410  007ECA  4A0B               	infsnz	main@x^0,f,c
   411  007ECC  2A0C               	incf	(main@x+1)^0,f,c
   412  007ECE                     
   413                           ;ADC.c: 45:         delay(10000);
   414  007ECE  0E27               	movlw	39
   415  007ED0  6E02               	movwf	(delay@ms+1)^0,c
   416  007ED2  0E10               	movlw	16
   417  007ED4  6E01               	movwf	delay@ms^0,c
   418  007ED6  ECEA  F03D         	call	_delay	;wreg free
   419  007EDA                     
   420                           ;ADC.c: 46:         delay(10000);
   421  007EDA  0E27               	movlw	39
   422  007EDC  6E02               	movwf	(delay@ms+1)^0,c
   423  007EDE  0E10               	movlw	16
   424  007EE0  6E01               	movwf	delay@ms^0,c
   425  007EE2  ECEA  F03D         	call	_delay	;wreg free
   426  007EE6                     
   427                           ;ADC.c: 47:         delay(10000);
   428  007EE6  0E27               	movlw	39
   429  007EE8  6E02               	movwf	(delay@ms+1)^0,c
   430  007EEA  0E10               	movlw	16
   431  007EEC  6E01               	movwf	delay@ms^0,c
   432  007EEE  ECEA  F03D         	call	_delay	;wreg free
   433  007EF2                     
   434                           ;ADC.c: 48:         command(0x01);
   435  007EF2  0E01               	movlw	1
   436  007EF4  ECC4  F03D         	call	_command
   437  007EF8  EFDC  F03E         	goto	l1029
   438  007EFC  EF00  F000         	goto	start
   439  007F00                     __end_of_main:
   440                           	callstack 0
   441                           
   442 ;; *************** function _data *****************
   443 ;; Defined at:
   444 ;;		line 55 in file "ADC.c"
   445 ;; Parameters:    Size  Location     Type
   446 ;;  b               1    wreg     unsigned char 
   447 ;; Auto vars:     Size  Location     Type
   448 ;;  b               1    5[COMRAM] unsigned char 
   449 ;; Return value:  Size  Location     Type
   450 ;;                  1    wreg      void 
   451 ;; Registers used:
   452 ;;		wreg, status,2, status,0, cstack
   453 ;; Tracked objects:
   454 ;;		On entry : 0/0
   455 ;;		On exit  : 0/0
   456 ;;		Unchanged: 0/0
   457 ;; Data sizes:     COMRAM   BANK0   BANK1   BANK2   BANK3   BANK4   BANK5
   458 ;;      Params:         0       0       0       0       0       0       0
   459 ;;      Locals:         1       0       0       0       0       0       0
   460 ;;      Temps:          0       0       0       0       0       0       0
   461 ;;      Totals:         1       0       0       0       0       0       0
   462 ;;Total ram usage:        1 bytes
   463 ;; Hardware stack levels used: 1
   464 ;; Hardware stack levels required when called: 1
   465 ;; This function calls:
   466 ;;		_delay
   467 ;; This function is called by:
   468 ;;		_main
   469 ;;		_display
   470 ;; This function uses a non-reentrant model
   471 ;;
   472                           
   473                           	psect	text1
   474  007BAE                     __ptext1:
   475                           	callstack 0
   476  007BAE                     _data:
   477                           	callstack 29
   478                           
   479                           ;incstack = 0
   480                           ;data@b stored from wreg
   481  007BAE  6E06               	movwf	data@b^0,c
   482  007BB0                     
   483                           ;ADC.c: 56:     PORTD=b;
   484  007BB0  C006  FF83         	movff	data@b,3971	;volatile
   485  007BB4                     
   486                           ;ADC.c: 57:     RC0=1;
   487  007BB4  8082               	bsf	3970,0,c	;volatile
   488  007BB6                     
   489                           ;ADC.c: 58:     RC1=1;
   490  007BB6  8282               	bsf	3970,1,c	;volatile
   491  007BB8                     
   492                           ;ADC.c: 59:     delay(1000);
   493  007BB8  0E03               	movlw	3
   494  007BBA  6E02               	movwf	(delay@ms+1)^0,c
   495  007BBC  0EE8               	movlw	232
   496  007BBE  6E01               	movwf	delay@ms^0,c
   497  007BC0  ECEA  F03D         	call	_delay	;wreg free
   498  007BC4                     
   499                           ;ADC.c: 60:     RC1=0;
   500  007BC4  9282               	bcf	3970,1,c	;volatile
   501  007BC6                     
   502                           ;ADC.c: 61:     delay(1000);
   503  007BC6  0E03               	movlw	3
   504  007BC8  6E02               	movwf	(delay@ms+1)^0,c
   505  007BCA  0EE8               	movlw	232
   506  007BCC  6E01               	movwf	delay@ms^0,c
   507  007BCE  ECEA  F03D         	call	_delay	;wreg free
   508  007BD2  0012               	return		;funcret
   509  007BD4                     __end_of_data:
   510                           	callstack 0
   511                           
   512 ;; *************** function _command *****************
   513 ;; Defined at:
   514 ;;		line 63 in file "ADC.c"
   515 ;; Parameters:    Size  Location     Type
   516 ;;  c               1    wreg     unsigned char 
   517 ;; Auto vars:     Size  Location     Type
   518 ;;  c               1    5[COMRAM] unsigned char 
   519 ;; Return value:  Size  Location     Type
   520 ;;                  1    wreg      void 
   521 ;; Registers used:
   522 ;;		wreg, status,2, status,0, cstack
   523 ;; Tracked objects:
   524 ;;		On entry : 0/0
   525 ;;		On exit  : 0/0
   526 ;;		Unchanged: 0/0
   527 ;; Data sizes:     COMRAM   BANK0   BANK1   BANK2   BANK3   BANK4   BANK5
   528 ;;      Params:         0       0       0       0       0       0       0
   529 ;;      Locals:         1       0       0       0       0       0       0
   530 ;;      Temps:          0       0       0       0       0       0       0
   531 ;;      Totals:         1       0       0       0       0       0       0
   532 ;;Total ram usage:        1 bytes
   533 ;; Hardware stack levels used: 1
   534 ;; Hardware stack levels required when called: 1
   535 ;; This function calls:
   536 ;;		_delay
   537 ;; This function is called by:
   538 ;;		_main
   539 ;; This function uses a non-reentrant model
   540 ;;
   541                           
   542                           	psect	text2
   543  007B88                     __ptext2:
   544                           	callstack 0
   545  007B88                     _command:
   546                           	callstack 29
   547                           
   548                           ;incstack = 0
   549                           ;command@c stored from wreg
   550  007B88  6E06               	movwf	command@c^0,c
   551  007B8A                     
   552                           ;ADC.c: 64:     PORTD=c;
   553  007B8A  C006  FF83         	movff	command@c,3971	;volatile
   554  007B8E                     
   555                           ;ADC.c: 65:     RC0=0;
   556  007B8E  9082               	bcf	3970,0,c	;volatile
   557  007B90                     
   558                           ;ADC.c: 66:     RC1=1;
   559  007B90  8282               	bsf	3970,1,c	;volatile
   560  007B92                     
   561                           ;ADC.c: 67:     delay(1000);
   562  007B92  0E03               	movlw	3
   563  007B94  6E02               	movwf	(delay@ms+1)^0,c
   564  007B96  0EE8               	movlw	232
   565  007B98  6E01               	movwf	delay@ms^0,c
   566  007B9A  ECEA  F03D         	call	_delay	;wreg free
   567  007B9E                     
   568                           ;ADC.c: 68:     RC1=0;
   569  007B9E  9282               	bcf	3970,1,c	;volatile
   570  007BA0                     
   571                           ;ADC.c: 69:     delay(1000);
   572  007BA0  0E03               	movlw	3
   573  007BA2  6E02               	movwf	(delay@ms+1)^0,c
   574  007BA4  0EE8               	movlw	232
   575  007BA6  6E01               	movwf	delay@ms^0,c
   576  007BA8  ECEA  F03D         	call	_delay	;wreg free
   577  007BAC  0012               	return		;funcret
   578  007BAE                     __end_of_command:
   579                           	callstack 0
   580                           
   581 ;; *************** function _delay *****************
   582 ;; Defined at:
   583 ;;		line 77 in file "ADC.c"
   584 ;; Parameters:    Size  Location     Type
   585 ;;  ms              2    0[COMRAM] int 
   586 ;; Auto vars:     Size  Location     Type
   587 ;;  i               2    3[COMRAM] int 
   588 ;; Return value:  Size  Location     Type
   589 ;;                  1    wreg      void 
   590 ;; Registers used:
   591 ;;		wreg, status,2, status,0
   592 ;; Tracked objects:
   593 ;;		On entry : 0/0
   594 ;;		On exit  : 0/0
   595 ;;		Unchanged: 0/0
   596 ;; Data sizes:     COMRAM   BANK0   BANK1   BANK2   BANK3   BANK4   BANK5
   597 ;;      Params:         2       0       0       0       0       0       0
   598 ;;      Locals:         2       0       0       0       0       0       0
   599 ;;      Temps:          1       0       0       0       0       0       0
   600 ;;      Totals:         5       0       0       0       0       0       0
   601 ;;Total ram usage:        5 bytes
   602 ;; Hardware stack levels used: 1
   603 ;; This function calls:
   604 ;;		Nothing
   605 ;; This function is called by:
   606 ;;		_main
   607 ;;		_data
   608 ;;		_command
   609 ;; This function uses a non-reentrant model
   610 ;;
   611                           
   612                           	psect	text3
   613  007BD4                     __ptext3:
   614                           	callstack 0
   615  007BD4                     _delay:
   616                           	callstack 30
   617  007BD4                     
   618                           ;ADC.c: 78:     for (int i=0;i<=ms;i++){
   619  007BD4  0E00               	movlw	0
   620  007BD6  6E05               	movwf	(delay@i+1)^0,c
   621  007BD8  0E00               	movlw	0
   622  007BDA  6E04               	movwf	delay@i^0,c
   623  007BDC  EFF2  F03D         	goto	l909
   624  007BE0                     l907:
   625                           
   626                           ;ADC.c: 80:     }
   627  007BE0  4A04               	infsnz	delay@i^0,f,c
   628  007BE2  2A05               	incf	(delay@i+1)^0,f,c
   629  007BE4                     l909:
   630  007BE4  5004               	movf	delay@i^0,w,c
   631  007BE6  5C01               	subwf	delay@ms^0,w,c
   632  007BE8  5002               	movf	(delay@ms+1)^0,w,c
   633  007BEA  0A80               	xorlw	128
   634  007BEC  6E03               	movwf	??_delay^0,c
   635  007BEE  5005               	movf	(delay@i+1)^0,w,c
   636  007BF0  0A80               	xorlw	128
   637  007BF2  5803               	subwfb	??_delay^0,w,c
   638  007BF4  B0D8               	btfsc	status,0,c
   639  007BF6  EFFF  F03D         	goto	u151
   640  007BFA  EF01  F03E         	goto	u150
   641  007BFE                     u151:
   642  007BFE  EFF0  F03D         	goto	l907
   643  007C02                     u150:
   644  007C02  0012               	return		;funcret
   645  007C04                     __end_of_delay:
   646                           	callstack 0
   647                           
   648 ;; *************** function ___awmod *****************
   649 ;; Defined at:
   650 ;;		line 7 in file "C:\Program Files\Microchip\xc8\v2.32\pic\sources\c99\common\awmod.c"
   651 ;; Parameters:    Size  Location     Type
   652 ;;  dividend        2    0[COMRAM] int 
   653 ;;  divisor         2    2[COMRAM] int 
   654 ;; Auto vars:     Size  Location     Type
   655 ;;  sign            1    5[COMRAM] unsigned char 
   656 ;;  counter         1    4[COMRAM] unsigned char 
   657 ;; Return value:  Size  Location     Type
   658 ;;                  2    0[COMRAM] int 
   659 ;; Registers used:
   660 ;;		wreg, status,2, status,0
   661 ;; Tracked objects:
   662 ;;		On entry : 0/0
   663 ;;		On exit  : 0/0
   664 ;;		Unchanged: 0/0
   665 ;; Data sizes:     COMRAM   BANK0   BANK1   BANK2   BANK3   BANK4   BANK5
   666 ;;      Params:         4       0       0       0       0       0       0
   667 ;;      Locals:         2       0       0       0       0       0       0
   668 ;;      Temps:          0       0       0       0       0       0       0
   669 ;;      Totals:         6       0       0       0       0       0       0
   670 ;;Total ram usage:        6 bytes
   671 ;; Hardware stack levels used: 1
   672 ;; This function calls:
   673 ;;		Nothing
   674 ;; This function is called by:
   675 ;;		_main
   676 ;; This function uses a non-reentrant model
   677 ;;
   678                           
   679                           	psect	text4
   680  007C04                     __ptext4:
   681                           	callstack 0
   682  007C04                     ___awmod:
   683                           	callstack 30
   684  007C04  0E00               	movlw	0
   685  007C06  6E06               	movwf	___awmod@sign^0,c
   686  007C08  BE02               	btfsc	(___awmod@dividend+1)^0,7,c
   687  007C0A  EF0B  F03E         	goto	u220
   688  007C0E  EF09  F03E         	goto	u221
   689  007C12                     u221:
   690  007C12  EF11  F03E         	goto	l987
   691  007C16                     u220:
   692  007C16  6C01               	negf	___awmod@dividend^0,c
   693  007C18  1E02               	comf	(___awmod@dividend+1)^0,f,c
   694  007C1A  B0D8               	btfsc	status,0,c
   695  007C1C  2A02               	incf	(___awmod@dividend+1)^0,f,c
   696  007C1E  0E01               	movlw	1
   697  007C20  6E06               	movwf	___awmod@sign^0,c
   698  007C22                     l987:
   699  007C22  BE04               	btfsc	(___awmod@divisor+1)^0,7,c
   700  007C24  EF18  F03E         	goto	u230
   701  007C28  EF16  F03E         	goto	u231
   702  007C2C                     u231:
   703  007C2C  EF1C  F03E         	goto	l991
   704  007C30                     u230:
   705  007C30  6C03               	negf	___awmod@divisor^0,c
   706  007C32  1E04               	comf	(___awmod@divisor+1)^0,f,c
   707  007C34  B0D8               	btfsc	status,0,c
   708  007C36  2A04               	incf	(___awmod@divisor+1)^0,f,c
   709  007C38                     l991:
   710  007C38  5003               	movf	___awmod@divisor^0,w,c
   711  007C3A  1004               	iorwf	(___awmod@divisor+1)^0,w,c
   712  007C3C  B4D8               	btfsc	status,2,c
   713  007C3E  EF23  F03E         	goto	u241
   714  007C42  EF25  F03E         	goto	u240
   715  007C46                     u241:
   716  007C46  EF49  F03E         	goto	l1007
   717  007C4A                     u240:
   718  007C4A  0E01               	movlw	1
   719  007C4C  6E05               	movwf	___awmod@counter^0,c
   720  007C4E  EF2D  F03E         	goto	l997
   721  007C52                     l995:
   722  007C52  90D8               	bcf	status,0,c
   723  007C54  3603               	rlcf	___awmod@divisor^0,f,c
   724  007C56  3604               	rlcf	(___awmod@divisor+1)^0,f,c
   725  007C58  2A05               	incf	___awmod@counter^0,f,c
   726  007C5A                     l997:
   727  007C5A  AE04               	btfss	(___awmod@divisor+1)^0,7,c
   728  007C5C  EF32  F03E         	goto	u251
   729  007C60  EF34  F03E         	goto	u250
   730  007C64                     u251:
   731  007C64  EF29  F03E         	goto	l995
   732  007C68                     u250:
   733  007C68                     l999:
   734  007C68  5003               	movf	___awmod@divisor^0,w,c
   735  007C6A  5C01               	subwf	___awmod@dividend^0,w,c
   736  007C6C  5004               	movf	(___awmod@divisor+1)^0,w,c
   737  007C6E  5802               	subwfb	(___awmod@dividend+1)^0,w,c
   738  007C70  A0D8               	btfss	status,0,c
   739  007C72  EF3D  F03E         	goto	u261
   740  007C76  EF3F  F03E         	goto	u260
   741  007C7A                     u261:
   742  007C7A  EF43  F03E         	goto	l1003
   743  007C7E                     u260:
   744  007C7E  5003               	movf	___awmod@divisor^0,w,c
   745  007C80  5E01               	subwf	___awmod@dividend^0,f,c
   746  007C82  5004               	movf	(___awmod@divisor+1)^0,w,c
   747  007C84  5A02               	subwfb	(___awmod@dividend+1)^0,f,c
   748  007C86                     l1003:
   749  007C86  90D8               	bcf	status,0,c
   750  007C88  3204               	rrcf	(___awmod@divisor+1)^0,f,c
   751  007C8A  3203               	rrcf	___awmod@divisor^0,f,c
   752  007C8C  2E05               	decfsz	___awmod@counter^0,f,c
   753  007C8E  EF34  F03E         	goto	l999
   754  007C92                     l1007:
   755  007C92  5006               	movf	___awmod@sign^0,w,c
   756  007C94  B4D8               	btfsc	status,2,c
   757  007C96  EF4F  F03E         	goto	u271
   758  007C9A  EF51  F03E         	goto	u270
   759  007C9E                     u271:
   760  007C9E  EF55  F03E         	goto	l1011
   761  007CA2                     u270:
   762  007CA2  6C01               	negf	___awmod@dividend^0,c
   763  007CA4  1E02               	comf	(___awmod@dividend+1)^0,f,c
   764  007CA6  B0D8               	btfsc	status,0,c
   765  007CA8  2A02               	incf	(___awmod@dividend+1)^0,f,c
   766  007CAA                     l1011:
   767  007CAA  C001  F001         	movff	___awmod@dividend,?___awmod
   768  007CAE  C002  F002         	movff	___awmod@dividend+1,?___awmod+1
   769  007CB2  0012               	return		;funcret
   770  007CB4                     __end_of___awmod:
   771                           	callstack 0
   772                           
   773 ;; *************** function ___awdiv *****************
   774 ;; Defined at:
   775 ;;		line 7 in file "C:\Program Files\Microchip\xc8\v2.32\pic\sources\c99\common\awdiv.c"
   776 ;; Parameters:    Size  Location     Type
   777 ;;  dividend        2    0[COMRAM] int 
   778 ;;  divisor         2    2[COMRAM] int 
   779 ;; Auto vars:     Size  Location     Type
   780 ;;  quotient        2    6[COMRAM] int 
   781 ;;  sign            1    5[COMRAM] unsigned char 
   782 ;;  counter         1    4[COMRAM] unsigned char 
   783 ;; Return value:  Size  Location     Type
   784 ;;                  2    0[COMRAM] int 
   785 ;; Registers used:
   786 ;;		wreg, status,2, status,0
   787 ;; Tracked objects:
   788 ;;		On entry : 0/0
   789 ;;		On exit  : 0/0
   790 ;;		Unchanged: 0/0
   791 ;; Data sizes:     COMRAM   BANK0   BANK1   BANK2   BANK3   BANK4   BANK5
   792 ;;      Params:         4       0       0       0       0       0       0
   793 ;;      Locals:         4       0       0       0       0       0       0
   794 ;;      Temps:          0       0       0       0       0       0       0
   795 ;;      Totals:         8       0       0       0       0       0       0
   796 ;;Total ram usage:        8 bytes
   797 ;; Hardware stack levels used: 1
   798 ;; This function calls:
   799 ;;		Nothing
   800 ;; This function is called by:
   801 ;;		_main
   802 ;; This function uses a non-reentrant model
   803 ;;
   804                           
   805                           	psect	text5
   806  007CB4                     __ptext5:
   807                           	callstack 0
   808  007CB4                     ___awdiv:
   809                           	callstack 30
   810  007CB4  0E00               	movlw	0
   811  007CB6  6E06               	movwf	___awdiv@sign^0,c
   812  007CB8  BE04               	btfsc	(___awdiv@divisor+1)^0,7,c
   813  007CBA  EF63  F03E         	goto	u160
   814  007CBE  EF61  F03E         	goto	u161
   815  007CC2                     u161:
   816  007CC2  EF69  F03E         	goto	l943
   817  007CC6                     u160:
   818  007CC6  6C03               	negf	___awdiv@divisor^0,c
   819  007CC8  1E04               	comf	(___awdiv@divisor+1)^0,f,c
   820  007CCA  B0D8               	btfsc	status,0,c
   821  007CCC  2A04               	incf	(___awdiv@divisor+1)^0,f,c
   822  007CCE  0E01               	movlw	1
   823  007CD0  6E06               	movwf	___awdiv@sign^0,c
   824  007CD2                     l943:
   825  007CD2  BE02               	btfsc	(___awdiv@dividend+1)^0,7,c
   826  007CD4  EF70  F03E         	goto	u170
   827  007CD8  EF6E  F03E         	goto	u171
   828  007CDC                     u171:
   829  007CDC  EF76  F03E         	goto	l949
   830  007CE0                     u170:
   831  007CE0  6C01               	negf	___awdiv@dividend^0,c
   832  007CE2  1E02               	comf	(___awdiv@dividend+1)^0,f,c
   833  007CE4  B0D8               	btfsc	status,0,c
   834  007CE6  2A02               	incf	(___awdiv@dividend+1)^0,f,c
   835  007CE8  0E01               	movlw	1
   836  007CEA  1A06               	xorwf	___awdiv@sign^0,f,c
   837  007CEC                     l949:
   838  007CEC  0E00               	movlw	0
   839  007CEE  6E08               	movwf	(___awdiv@quotient+1)^0,c
   840  007CF0  0E00               	movlw	0
   841  007CF2  6E07               	movwf	___awdiv@quotient^0,c
   842  007CF4  5003               	movf	___awdiv@divisor^0,w,c
   843  007CF6  1004               	iorwf	(___awdiv@divisor+1)^0,w,c
   844  007CF8  B4D8               	btfsc	status,2,c
   845  007CFA  EF81  F03E         	goto	u181
   846  007CFE  EF83  F03E         	goto	u180
   847  007D02                     u181:
   848  007D02  EFAB  F03E         	goto	l971
   849  007D06                     u180:
   850  007D06  0E01               	movlw	1
   851  007D08  6E05               	movwf	___awdiv@counter^0,c
   852  007D0A  EF8B  F03E         	goto	l957
   853  007D0E                     l955:
   854  007D0E  90D8               	bcf	status,0,c
   855  007D10  3603               	rlcf	___awdiv@divisor^0,f,c
   856  007D12  3604               	rlcf	(___awdiv@divisor+1)^0,f,c
   857  007D14  2A05               	incf	___awdiv@counter^0,f,c
   858  007D16                     l957:
   859  007D16  AE04               	btfss	(___awdiv@divisor+1)^0,7,c
   860  007D18  EF90  F03E         	goto	u191
   861  007D1C  EF92  F03E         	goto	u190
   862  007D20                     u191:
   863  007D20  EF87  F03E         	goto	l955
   864  007D24                     u190:
   865  007D24                     l959:
   866  007D24  90D8               	bcf	status,0,c
   867  007D26  3607               	rlcf	___awdiv@quotient^0,f,c
   868  007D28  3608               	rlcf	(___awdiv@quotient+1)^0,f,c
   869  007D2A  5003               	movf	___awdiv@divisor^0,w,c
   870  007D2C  5C01               	subwf	___awdiv@dividend^0,w,c
   871  007D2E  5004               	movf	(___awdiv@divisor+1)^0,w,c
   872  007D30  5802               	subwfb	(___awdiv@dividend+1)^0,w,c
   873  007D32  A0D8               	btfss	status,0,c
   874  007D34  EF9E  F03E         	goto	u201
   875  007D38  EFA0  F03E         	goto	u200
   876  007D3C                     u201:
   877  007D3C  EFA5  F03E         	goto	l967
   878  007D40                     u200:
   879  007D40  5003               	movf	___awdiv@divisor^0,w,c
   880  007D42  5E01               	subwf	___awdiv@dividend^0,f,c
   881  007D44  5004               	movf	(___awdiv@divisor+1)^0,w,c
   882  007D46  5A02               	subwfb	(___awdiv@dividend+1)^0,f,c
   883  007D48  8007               	bsf	___awdiv@quotient^0,0,c
   884  007D4A                     l967:
   885  007D4A  90D8               	bcf	status,0,c
   886  007D4C  3204               	rrcf	(___awdiv@divisor+1)^0,f,c
   887  007D4E  3203               	rrcf	___awdiv@divisor^0,f,c
   888  007D50  2E05               	decfsz	___awdiv@counter^0,f,c
   889  007D52  EF92  F03E         	goto	l959
   890  007D56                     l971:
   891  007D56  5006               	movf	___awdiv@sign^0,w,c
   892  007D58  B4D8               	btfsc	status,2,c
   893  007D5A  EFB1  F03E         	goto	u211
   894  007D5E  EFB3  F03E         	goto	u210
   895  007D62                     u211:
   896  007D62  EFB7  F03E         	goto	l975
   897  007D66                     u210:
   898  007D66  6C07               	negf	___awdiv@quotient^0,c
   899  007D68  1E08               	comf	(___awdiv@quotient+1)^0,f,c
   900  007D6A  B0D8               	btfsc	status,0,c
   901  007D6C  2A08               	incf	(___awdiv@quotient+1)^0,f,c
   902  007D6E                     l975:
   903  007D6E  C007  F001         	movff	___awdiv@quotient,?___awdiv
   904  007D72  C008  F002         	movff	___awdiv@quotient+1,?___awdiv+1
   905  007D76  0012               	return		;funcret
   906  007D78                     __end_of___awdiv:
   907                           	callstack 0
   908  0000                     
   909                           	psect	rparam
   910  0000                     
   911                           	psect	idloc
   912                           
   913                           ;Config register IDLOC0 @ 0x200000
   914                           ;	unspecified, using default values
   915  200000                     	org	2097152
   916  200000  FF                 	db	255
   917                           
   918                           ;Config register IDLOC1 @ 0x200001
   919                           ;	unspecified, using default values
   920  200001                     	org	2097153
   921  200001  FF                 	db	255
   922                           
   923                           ;Config register IDLOC2 @ 0x200002
   924                           ;	unspecified, using default values
   925  200002                     	org	2097154
   926  200002  FF                 	db	255
   927                           
   928                           ;Config register IDLOC3 @ 0x200003
   929                           ;	unspecified, using default values
   930  200003                     	org	2097155
   931  200003  FF                 	db	255
   932                           
   933                           ;Config register IDLOC4 @ 0x200004
   934                           ;	unspecified, using default values
   935  200004                     	org	2097156
   936  200004  FF                 	db	255
   937                           
   938                           ;Config register IDLOC5 @ 0x200005
   939                           ;	unspecified, using default values
   940  200005                     	org	2097157
   941  200005  FF                 	db	255
   942                           
   943                           ;Config register IDLOC6 @ 0x200006
   944                           ;	unspecified, using default values
   945  200006                     	org	2097158
   946  200006  FF                 	db	255
   947                           
   948                           ;Config register IDLOC7 @ 0x200007
   949                           ;	unspecified, using default values
   950  200007                     	org	2097159
   951  200007  FF                 	db	255
   952                           
   953                           	psect	config
   954                           
   955                           ; Padding undefined space
   956  300000                     	org	3145728
   957  300000  FF                 	db	255
   958                           
   959                           ;Config register CONFIG1H @ 0x300001
   960                           ;	unspecified, using default values
   961                           ;	Oscillator Selection bits
   962                           ;	OSC = 0x7, unprogrammed default
   963                           ;	Fail-Safe Clock Monitor Enable bit
   964                           ;	FCMEN = 0x0, unprogrammed default
   965                           ;	Internal/External Oscillator Switchover bit
   966                           ;	IESO = 0x0, unprogrammed default
   967  300001                     	org	3145729
   968  300001  07                 	db	7
   969                           
   970                           ;Config register CONFIG2L @ 0x300002
   971                           ;	unspecified, using default values
   972                           ;	Power-up Timer Enable bit
   973                           ;	PWRT = 0x1, unprogrammed default
   974                           ;	Brown-out Reset Enable bits
   975                           ;	BOREN = 0x3, unprogrammed default
   976                           ;	Brown-out Reset Voltage bits
   977                           ;	BORV = 0x3, unprogrammed default
   978  300002                     	org	3145730
   979  300002  1F                 	db	31
   980                           
   981                           ;Config register CONFIG2H @ 0x300003
   982                           ;	unspecified, using default values
   983                           ;	Watchdog Timer Enable bit
   984                           ;	WDT = 0x1, unprogrammed default
   985                           ;	Watchdog Timer Postscale Select bits
   986                           ;	WDTPS = 0xF, unprogrammed default
   987  300003                     	org	3145731
   988  300003  1F                 	db	31
   989                           
   990                           ; Padding undefined space
   991  300004                     	org	3145732
   992  300004  FF                 	db	255
   993                           
   994                           ;Config register CONFIG3H @ 0x300005
   995                           ;	unspecified, using default values
   996                           ;	PORTB A/D Enable bit
   997                           ;	PBADEN = 0x1, unprogrammed default
   998                           ;	Low-Power Timer 1 Oscillator Enable bit
   999                           ;	LPT1OSC = 0x0, unprogrammed default
  1000                           ;	MCLR Pin Enable bit
  1001                           ;	MCLRE = 0x1, unprogrammed default
  1002  300005                     	org	3145733
  1003  300005  82                 	db	130
  1004                           
  1005                           ;Config register CONFIG4L @ 0x300006
  1006                           ;	unspecified, using default values
  1007                           ;	Stack Full/Underflow Reset Enable bit
  1008                           ;	STVREN = 0x1, unprogrammed default
  1009                           ;	Single-Supply ICSP Enable bit
  1010                           ;	LVP = 0x1, unprogrammed default
  1011                           ;	Boot Block Size Select bit
  1012                           ;	BBSIZ = 0x0, unprogrammed default
  1013                           ;	Extended Instruction Set Enable bit
  1014                           ;	XINST = 0x0, unprogrammed default
  1015                           ;	Background Debugger Enable bit
  1016                           ;	DEBUG = 0x1, unprogrammed default
  1017  300006                     	org	3145734
  1018  300006  85                 	db	133
  1019                           
  1020                           ; Padding undefined space
  1021  300007                     	org	3145735
  1022  300007  FF                 	db	255
  1023                           
  1024                           ;Config register CONFIG5L @ 0x300008
  1025                           ;	unspecified, using default values
  1026                           ;	Code Protection bit
  1027                           ;	CP0 = 0x1, unprogrammed default
  1028                           ;	Code Protection bit
  1029                           ;	CP1 = 0x1, unprogrammed default
  1030                           ;	Code Protection bit
  1031                           ;	CP2 = 0x1, unprogrammed default
  1032                           ;	Code Protection bit
  1033                           ;	CP3 = 0x1, unprogrammed default
  1034  300008                     	org	3145736
  1035  300008  0F                 	db	15
  1036                           
  1037                           ;Config register CONFIG5H @ 0x300009
  1038                           ;	unspecified, using default values
  1039                           ;	Boot Block Code Protection bit
  1040                           ;	CPB = 0x1, unprogrammed default
  1041                           ;	Data EEPROM Code Protection bit
  1042                           ;	CPD = 0x1, unprogrammed default
  1043  300009                     	org	3145737
  1044  300009  C0                 	db	192
  1045                           
  1046                           ;Config register CONFIG6L @ 0x30000A
  1047                           ;	unspecified, using default values
  1048                           ;	Write Protection bit
  1049                           ;	WRT0 = 0x1, unprogrammed default
  1050                           ;	Write Protection bit
  1051                           ;	WRT1 = 0x1, unprogrammed default
  1052                           ;	Write Protection bit
  1053                           ;	WRT2 = 0x1, unprogrammed default
  1054                           ;	Write Protection bit
  1055                           ;	WRT3 = 0x1, unprogrammed default
  1056  30000A                     	org	3145738
  1057  30000A  0F                 	db	15
  1058                           
  1059                           ;Config register CONFIG6H @ 0x30000B
  1060                           ;	unspecified, using default values
  1061                           ;	Configuration Register Write Protection bit
  1062                           ;	WRTC = 0x1, unprogrammed default
  1063                           ;	Boot Block Write Protection bit
  1064                           ;	WRTB = 0x1, unprogrammed default
  1065                           ;	Data EEPROM Write Protection bit
  1066                           ;	WRTD = 0x1, unprogrammed default
  1067  30000B                     	org	3145739
  1068  30000B  E0                 	db	224
  1069                           
  1070                           ;Config register CONFIG7L @ 0x30000C
  1071                           ;	unspecified, using default values
  1072                           ;	Table Read Protection bit
  1073                           ;	EBTR0 = 0x1, unprogrammed default
  1074                           ;	Table Read Protection bit
  1075                           ;	EBTR1 = 0x1, unprogrammed default
  1076                           ;	Table Read Protection bit
  1077                           ;	EBTR2 = 0x1, unprogrammed default
  1078                           ;	Table Read Protection bit
  1079                           ;	EBTR3 = 0x1, unprogrammed default
  1080  30000C                     	org	3145740
  1081  30000C  0F                 	db	15
  1082                           
  1083                           ;Config register CONFIG7H @ 0x30000D
  1084                           ;	unspecified, using default values
  1085                           ;	Boot Block Table Read Protection bit
  1086                           ;	EBTRB = 0x1, unprogrammed default
  1087  30000D                     	org	3145741
  1088  30000D  40                 	db	64
  1089                           tosu	equ	0xFFF
  1090                           tosh	equ	0xFFE
  1091                           tosl	equ	0xFFD
  1092                           stkptr	equ	0xFFC
  1093                           pclatu	equ	0xFFB
  1094                           pclath	equ	0xFFA
  1095                           pcl	equ	0xFF9
  1096                           tblptru	equ	0xFF8
  1097                           tblptrh	equ	0xFF7
  1098                           tblptrl	equ	0xFF6
  1099                           tablat	equ	0xFF5
  1100                           prodh	equ	0xFF4
  1101                           prodl	equ	0xFF3
  1102                           indf0	equ	0xFEF
  1103                           postinc0	equ	0xFEE
  1104                           postdec0	equ	0xFED
  1105                           preinc0	equ	0xFEC
  1106                           plusw0	equ	0xFEB
  1107                           fsr0h	equ	0xFEA
  1108                           fsr0l	equ	0xFE9
  1109                           wreg	equ	0xFE8
  1110                           indf1	equ	0xFE7
  1111                           postinc1	equ	0xFE6
  1112                           postdec1	equ	0xFE5
  1113                           preinc1	equ	0xFE4
  1114                           plusw1	equ	0xFE3
  1115                           fsr1h	equ	0xFE2
  1116                           fsr1l	equ	0xFE1
  1117                           bsr	equ	0xFE0
  1118                           indf2	equ	0xFDF
  1119                           postinc2	equ	0xFDE
  1120                           postdec2	equ	0xFDD
  1121                           preinc2	equ	0xFDC
  1122                           plusw2	equ	0xFDB
  1123                           fsr2h	equ	0xFDA
  1124                           fsr2l	equ	0xFD9
  1125                           status	equ	0xFD8

Data Sizes:
    Strings     0
    Constant    0
    Data        0
    BSS         0
    Persistent  0
    Stack       0

Auto Spaces:
    Space          Size  Autos    Used
    COMRAM           95     24      24
    BANK0           160      0       0
    BANK1           256      0       0
    BANK2           256      0       0
    BANK3           256      0       0
    BANK4           256      0       0
    BANK5           256      0       0

Pointer List with Targets:

    None.

Critical Paths under _main in COMRAM

    _main->___awdiv
    _data->_delay
    _command->_delay

Critical Paths under _main in BANK0

    None.

Critical Paths under _main in BANK1

    None.

Critical Paths under _main in BANK2

    None.

Critical Paths under _main in BANK3

    None.

Critical Paths under _main in BANK4

    None.

Critical Paths under _main in BANK5

    None.

Call Graph Tables:

 ---------------------------------------------------------------------------------
 (Depth) Function   	        Calls       Base Space   Used Autos Params    Refs
 ---------------------------------------------------------------------------------
 (0) _main                                                16    16      0    3791
                                              8 COMRAM    16    16      0
                            ___awdiv
                            ___awmod
                            _command
                               _data
                              _delay
 ---------------------------------------------------------------------------------
 (1) _data                                                 1     1      0     676
                                              5 COMRAM     1     1      0
                              _delay
 ---------------------------------------------------------------------------------
 (1) _command                                              1     1      0     676
                                              5 COMRAM     1     1      0
                              _delay
 ---------------------------------------------------------------------------------
 (1) _delay                                                5     3      2     654
                                              0 COMRAM     5     3      2
 ---------------------------------------------------------------------------------
 (1) ___awmod                                              6     2      4     752
                                              0 COMRAM     6     2      4
 ---------------------------------------------------------------------------------
 (1) ___awdiv                                              8     4      4     756
                                              0 COMRAM     8     4      4
 ---------------------------------------------------------------------------------
 Estimated maximum stack depth 1
 ---------------------------------------------------------------------------------

 Call Graph Graphs:

 _main (ROOT)
   ___awdiv
   ___awmod
   _command
     _delay
   _data
     _delay
   _delay

 Address spaces:
Name               Size   Autos  Total    Cost      Usage
BITCOMRAM           5F      0       0       0        0.0%
EEDATA             100      0       0       0        0.0%
NULL                 0      0       0       0        0.0%
CODE                 0      0       0       0        0.0%
COMRAM              5F     18      18       1       25.3%
STACK                0      0       0       2        0.0%
ABS                  0      0       0       3        0.0%
BITBANK0            A0      0       0       4        0.0%
BANK0               A0      0       0       5        0.0%
BITBANK1           100      0       0       6        0.0%
BANK1              100      0       0       7        0.0%
BITBANK2           100      0       0       8        0.0%
BANK2              100      0       0       9        0.0%
BITBANK3           100      0       0      10        0.0%
BANK3              100      0       0      11        0.0%
BITBANK4           100      0       0      12        0.0%
BANK4              100      0       0      13        0.0%
BITBANK5           100      0       0      14        0.0%
BANK5              100      0       0      15        0.0%
BIGRAM             5FF      0       0      16        0.0%
DATA                 0      0       0      17        0.0%
BITSFR_3             0      0       0     200        0.0%
SFR_3                0      0       0     200        0.0%
BITSFR_2             0      0       0     200        0.0%
SFR_2                0      0       0     200        0.0%
BITSFR_1             0      0       0     200        0.0%
SFR_1                0      0       0     200        0.0%
BITSFR               0      0       0     200        0.0%
SFR                  0      0       0     200        0.0%


Microchip Technology PIC18 Macro Assembler V2.32 build 20210201212658 
Symbol Table                                                                                   Wed Jan 19 10:39:02 2022

                     l40 7DD2                       l61 7C02                       l46 7BD2  
                     l38 7DC4                       l49 7BAC             ___awdiv@sign 0006  
                    l308 7CB2                      l295 7D76                      l911 7B8A  
                    l905 7BD4                      l921 7BA0                      l913 7B8E  
                    l907 7BE0                      l915 7B90                      l931 7BC4  
                    l923 7BB0                      l941 7CCE                      l909 7BE4  
                    l917 7B92                      l933 7BC6                      l925 7BB4  
                    l951 7CF4                      l943 7CD2                      l935 7CB4  
                    l919 7B9E                      l927 7BB6                      l961 7D2A  
                    l953 7D06                      l945 7CE0                      l937 7CB8  
                    l929 7BB8                      l963 7D40                      l955 7D0E  
                    l971 7D56                      l947 7CE8                      l939 7CC6  
                    l973 7D66                      l965 7D48                      l957 7D16  
                    l949 7CEC                      l981 7C08                      l975 7D6E  
                    l967 7D4A                      l959 7D24                      l991 7C38  
                    l983 7C16                      l969 7D50                      l993 7C4A  
                    l985 7C1E                      l995 7C52                      l987 7C22  
                    l979 7C04                      l997 7C5A                      l989 7C30  
                    l999 7C68                      _RC0 007C10                      _RC1 007C11  
                    u200 7D40                      u201 7D3C                      u210 7D66  
                    u211 7D62                      u220 7C16                      u221 7C12  
                    u230 7C30                      u150 7C02                      u231 7C2C  
                    u151 7BFE                      u160 7CC6                      u240 7C4A  
                    u161 7CC2                      u241 7C46                      u170 7CE0  
                    u250 7C68                      u171 7CDC                      u251 7C64  
                    u180 7D06                      u260 7C7E                      u181 7D02  
                    u261 7C7A                      u190 7D24                      u270 7CA2  
                    u191 7D20                      u271 7C9E                      u280 7DD2  
                    u281 7DCE             ___awmod@sign 0006                     l1001 7C7E  
                   l1011 7CAA                     l1003 7C86                     l1005 7C8C  
                   l1021 7DA0                     l1007 7C92                     l1031 7DC2  
                   l1023 7DA6                     l1015 7D78                     l1009 7CA2  
                   l1041 7E16                     l1033 7DD8                     l1025 7DAC  
                   l1017 7D98                     l1051 7E7A                     l1043 7E32  
                   l1035 7DE6                     l1027 7DB2                     l1019 7D9A  
                   l1061 7ECA                     l1053 7E82                     l1045 7E3A  
                   l1037 7E02                     l1029 7DB8                     l1063 7ECE  
                   l1055 7E9E                     l1047 7E56                     l1039 7E0A  
                   l1065 7EDA                     l1057 7EA6                     l1049 7E5E  
                   l1067 7EE6                     l1059 7EC2                     l1069 7EF2  
                   _data 7BAE                     _main 7D78                     start 0000  
           ___param_bank 000000                    ?_data 0001                    ?_main 0001  
        __end_of___awdiv 7D78          __end_of___awmod 7CB4          ___awdiv@divisor 0003  
        ___awdiv@counter 0005                    _PORTD 000F83                    _TRISA 000F92  
                  _TRISB 000F93                    _TRISC 000F94                    _TRISD 000F95  
        __end_of_command 7BAE                    _delay 7BD4                    data@b 0006  
                  main@a 0013                    main@p 000D                    main@q 0015  
                  main@r 000F                    main@s 0011                    main@x 000B  
                  main@y 0017                    status 000FD8          __initialization 7B82  
           __end_of_data 7BD4             __end_of_main 7F00                   ??_data 0006  
                 ??_main 0009            __activetblptr 000000                   ?_delay 0001  
                 _ADCON0 000FC2                   _ADCON1 000FC1                   _ADCON2 000FC0  
                 _ADRESH 000FC4                   _ADRESL 000FC3         ___awdiv@dividend 0001  
                 _GODONE 007E11                ??___awdiv 0005                ??___awmod 0005  
                 delay@i 0004         ___awdiv@quotient 0007          ___awmod@divisor 0003  
                 isa$std 000001          ___awmod@counter 0005                ??_command 0006  
             __accesstop 0060  __end_of__initialization 7B82            ___rparam_used 000001  
         __pcstackCOMRAM 0001            __end_of_delay 7C04                  ??_delay 0003  
                __Hparam 0000                  __Lparam 0000                  ___awdiv 7CB4  
                ___awmod 7C04                  __pcinit 7B82                  __ramtop 0600  
                __ptext0 7D78                  __ptext1 7BAE                  __ptext2 7B88  
                __ptext3 7BD4                  __ptext4 7C04                  __ptext5 7CB4  
                _command 7B88                  delay@ms 0001         ___awmod@dividend 0001  
   end_of_initialization 7B82      start_initialization 7B82                 ?___awdiv 0001  
               ?___awmod 0001                 ?_command 0001           __size_of_delay 0030  
               __Hrparam 0000                 __Lrparam 0000         __size_of___awdiv 00C4  
       __size_of___awmod 00B0         __size_of_command 0026            __size_of_data 0026  
          __size_of_main 0188                 isa$xinst 000000                 command@c 0006  
